:1003C4005452414E5A005354414E44414C4F4E45B1
:1003D400000000112332465765748C9DAFBECADB02
:1003E400E9F810013322564775649C8DBFAEDACB11
:1003F400F9E82130021367764455ADBC8E9FEBFAC1
:10040400C8D93120120377665445BDAC9E8FFBEAF0
:10041400D8C94253617004152736CEDFEDFC8899A4
:10042400ABBA5243716014053726DECFFDEC9889D0
:10043400BBAA6372405125340617EFFECCDDA9B880
:100444008A9B7362504135241607FFEEDCCDB9A8B0
:100454009A8B8495A7B6C2D3E1F008192B3A4E5F64
:100464006D7C9485B7A6D2C3F1E018093B2A5E4F90
:100474007D6CA5B48697E3F2C0D129380A1B6F7E40
:100484004C5DB5A49687F3E2D0C139281A0B7F6E70
:100494005C4DC6D7E5F48091A3B24A5B69780C1D24
:1004A4002F3ED6C7F5E49081B3A25A4B79681C0D50
:1004B4003F2EE7F6C4D5A1B082936B7A48592D3C00
:1004C4000E1FF7E6D4C5B1A092837B6A58493D2C30
:1004D4001E0F0089129B24AD36BF48C15AD36CE568
:1004E4007EF78108931AA52CB73EC940DB52ED6410
:1004F400FF76028B109926AF34BD4AC358D16EE7FC
:100504007CF5830A9118A72EB53CCB42D950EF66EF
:10051400FD74048D169F20A932BB4CC55ED768E1DB
:100524007AF3850C971EA128B33ACD44DF56E960CF
:10053400FB72068F149D22AB30B94EC75CD56AE3BB
:1005440078F1870E951CA32AB138CF46DD54EB62AF
:10055400F97008811A932CA53EB740C952DB64EDAB
:1005640076FF89009B12AD24BF36C148D35AE56C8F
:10057400F77E0A8318912EA73CB542CB50D966EF7B
:1005840074FD8B029910AF26BD34C34AD158E76E6F
:10059400F57C0C851E9728A13AB344CD56DF60E95B
:1005A40072FB8D049F16A920BB32C54CD75EE1684F
:1005B400F37A0E871C952AA338B146CF54DD62EB3B
:1005C40070F98F069D14AB22B930C74ED55CE36A2F
:0B05D400F178FF03C4FF03CAFF03D54A
:0319E70001760086
:10192C009001F2E06FFC9004D693FE9001F0E0FD84
:10193C00EE6D9001F2F0AF04EF9003D6939001F0AE
:01194C00F0AA
:01194D002277
:10000300C2AFC28E758900438910758BE0758DC1AF
:07001300D2ABD28ED2AF2266
:03001B0002177D4C
:10177D00C0E0C0D0C28E758BE0758DC1201B067583
:10178D00A61E75A6E10576D218E57C6002057C05DE
:10179D007FE57F540F7020D223E57F543F7002D236
:1017AD0014E57BD394014002157BE57ED394644010
:0E17BD0004D21B8002057ED28ED0D0D0E03246
:030023000212B016
:0B12B000C0E0C083C082C0D075D01821
:1012BB00309850757C01AF99201709EF640270418B
:1012CB00D217803D301F04C21F8024BF0904D21FD8
:1012DB00802FBF02055378808027BF031290002216
:1012EB00E578F0637840537840C217D21A801274B5
:1012FB006F2578F582E43401F583EFF005785378A8
:10130B007FC298309964C29930165F9000A6E0FFB7
:10131B009000EDE0D39F400DC216D220201D02D2CB
:10132B0021C21D80459000EDE0FF04F074EE2FF517
:10133B0082E43400F583E0F57D301C16537D7F305D
:10134B00152520D00520191F800330191A637D80C5
:10135B008015301512E57D527D301906A2D0929B77
:0C136B008005A2D0B3929B857D99D2AF83
:09137700D0D0D082D083D0E03246
:10187D00C216C221C21AC217C21FE49000EDF09029
:10188D0000A6F0F578F57CC21CD220E579F5CBE504
:0E189D007AF5CA85CBCD85CACCD29CD2AC22BE
:0610F9007E007F007D0275
:0210FF00A90541
:10110100E49001F0F09001F2F08E4E8F4F9000EEDE
:101111007402F0E4FB7A01EBC3995051854F82854B
:101121004E83E0FF12192C854F82854E83E024FD0A
:10113100600824FA600424077010AF020A74EE2FCD
:10114100F582E43400F5837409F0054FE54FAE4EA6
:101151007002054E14F5828E83E0FFAE020A74EE32
:101161002EF582E43400F583EFF00B80AA9001F2B2
:10117100E0FF24FD600824FA600424077010AE0229
:101181000A74EE2EF582E43400F5837409F0AE02A0
:101191000A74EE2EF582E43400F583EFF09001F04D
:1011A100E0FF24FD600824FA600424077010AE02F9
:1011B1000A74EE2EF582E43400F5837409F0AE0270
:1011C1000A74EE2EF582E43400F583EFF074EE2A12
:0C11D100F582E43400F5837403F0AF02F3
:0111DD0022EF
:10181200E49001F0F09001F2F0900022E05440FBDD
:10182200900022E0FFEBC39F5012746F2BF582E40D
:101832003401F583E0FF12192C0B80E49001F0E0F3
:0B184200FF9001F2E04F7002C322D3C0
:01184D002278
:10003600C2AF1217CBD2AFC2221211DE12187DC286
:100046001B120003C2AFE49001F1F0757B01D2AF41
:1000560075A70775A61E75A6E102035A302323C2AB
:10006600239001EFE0600B14F0E07006E577600284
:1000760015779001F3E0600214F09001F1E0600260
:1000860014F0E4F57E201E030202341207D7900016
:10009600A7E024FE700302019414700302021A14EE
:1000A60070030201CB1470030201F2240470AD1236
:1000B600184E9000A8EFF0600302018B900022E03A
:1000C600700302016412181250030202B290002259
:1000D600E0FF5440FEF54DFD054D746F2DF582E4AD
:1000E6003401F583E09000A5F0E0B4FE04C2AF80D1
:1000F600FE202210746F254DF582E43401F583E06D
:1001060090016EF0054DEF543FFFD39404404474C4
:100116006F2EF582E43401F58363A2019000246317
:10012600A201EF14FF121045900022E0543F24FC78
:10013600FF9000A4F012196F9000A7500B7404F002
:100146009001F37414F080137405F09001F3740FAA
:10015600F08008E49001EFF075770A0202B2900190
:10016600F1E060030200627425F01213803022036E
:100176000200629000A5E090020CF0A374FDF090DE
:1001860000A87414F09000A77402F0020062301602
:1001960003020062E49001F0F09001F2F07E027F2B
:1001A6000C9000A8E0FD1210FF9000A6EFF0E4907E
:1001B60000EDF0D216D2999000A704F09001EF74EA
:1001C60006F00200629000A4E0FF12196F400F9043
:1001D60000A77405F09001F3740FF002006290011D
:1001E600F3E06003020062C2AF020062120026EF73
:1001F60060169000A5E0900000F090016EE090007F
:1002060001F09000A77403F09001F3E06003020090
:10021600620203863016030200621210F99000A6ED
:10022600EFF0E49000EDF0D216D29902038690002A
:1002360023E024FE606814700302038E1470030228
:1002460003622403600302006230220E12194ED2AA
:100256001E9000A77401F0020062301603020062CD
:1002660090000074FEF0A374A0F0A37431F0A374A0
:100276002EF0A37430F0A3F07E007F007D061210EE
:10028600FF9000A6EFF0E49000EDF0D216D2999020
:1002960000237402F09001EF740AF00200629000ED
:1002A60022E070030203511218125008E490002253
:1002B600F0020062900022E0FF5440F54DFE054D2D
:1002C600746F2EF582E43401F583E09000A5F020EA
:1002D6002210746F254DF582E43401F583E0900118
:1002E6006EF0EF543FD3940A404090016EE0649064
:1002F6007038F54D7424254DF582E43400F5837489
:1003060020F0054DE54DB480EB900022E0FF54400F
:100316002471F582E43401F58363A201900024631D
:10032600A201EF543F14FF121045E4900022F09012
:10033600016EE0B4900C12194E9000237404F00282
:1003460000629000237403F00200629001EFE06007
:100356000302006290002304F002006230160302DA
:100366000062121A138F4D7E027F0CAD4D1210FFE4
:100376009000A6EFF0E49000EDF0D216D299D21ECE
:100386009000A704F002006230160302006290009B
:10039600A5E0900000F090016EE0900001F01210D0
:1003A600F99000A6EFF0E49000EDF0D216D2999005
:0E03B60000237402F09001EF740AF00200625E
:1011DE00E4F54EE54E75F003A424D6F582E434050D
:1011EE00F583E493FB740193FA740293F91205DF0D
:1011FE0070030212AFE4F550F551F54F7424254FEC
:10120E00F582E43400F583E0FF70030212AAE54E86
:10121E0075F003A424D6F582E43405F583E493FB3C
:10122E00740193FA740293F9855082758300120546
:10123E00F8FEEFB506077551010550805AE551606D
:10124E0056EE704EE54E1460450470507424254FD2
:10125E00F9E43400FA7B01C0031B8B59755A0075F3
:10126E005B00E4F55CD0031209878F558E548D53C5
:10127E008C52AB55AA54A953A8527FB07E717D0BE8
:10128E007C001206611206F38E798F7A800ED222BE
:10129E00800AE4F551F550054F02120A054E02116F
:0112AE00E15E
:0112AF00221C
:1014DA0042415544004E4F5F4D45414E44520057DC
:1014EA005F4D4F44454D00534C415645004C4541D4
:1014FA0044455200494E565F52454300494E565F95
:10150A005452414E5300494E565F414C4C0000C85C
:10151A00CCDF73696E7573625F6772616E69742E70
:10152A0062696E00312E3000C4C0D2C031312F3210
:10153A00392F31300031303A32323A303800FF1424
:10154A00DAFF14DFFF14E9FF14F1FF14F7FF14FEAA
:10155A00FF1506FF1510FF15180008040C020A06ED
:09156A000E0109050D030B070F2A
:1019EA005201F800000000000000000000000000A2
:0519FA000000000000E8
:061A1300900310E0FF2229
:100CC900E4900310F0E0FF04F0740C2FF582E43493
:100CD90002F58374FEF0900310E0FF04F0740C2F0A
:100CE900F582E43402F5837491F0900310E0FF0477
:100CF900F0740C2FF582E43402F5837430F090031C
:100D090010E0FF04F0740C2FF582E43402F58374CB
:100D19000DF0900310E0FF04F0740C2FF582E43419
:100D290002F583740AF0E4FFEFC39404501EEF90B8
:100D3900152E93FE900310E0240CF582E43402F59D
:100D490083EEF00F900310E004F080DCE4FFEFC3C2
:100D59009415501EEF90151C93FE900310E0240C7F
:100D6900F582E43402F583EEF00F900310E004F00D
:100D790080DCE4FFEFC3940D501EEF90153693FE0F
:100D8900900310E0240CF582E43402F583EEF00FB1
:100D9900900310E004F080DC900310E0FF04F0748D
:100DA9000C2FF582E43402F5837420F0E4FFEFC3DD
:100DB9009409501EEF90153F93FE900310E0240C08
:100DC900F582E43402F583EEF00F900310E004F0AD
:100DD90080DC900310E0FF04F0740C2FF582E434FA
:100DE90002F583740AF0900310E0FF04F0740C2FED
:090DF900F582E43402F583E4F014
:010E020022CD
:1019900090030EE06FFC9004D693FE90030FE06E70
:0F19A00090030EF0AF04EF9003D69390030FF077
:0119AF002215
:021674008F568F
:10167600900310E0240CF582E43402F5837420F024
:10168600900310E004F0E4FFEFC39D503BE5567570
:10169600F003A42448F582E43415F583E493FB743F
:1016A6000193FA740293F98F827583001205F8FE8E
:1016B600900310E0240CF582E43402F583EEF00F7B
:0816C600900310E004F080C065
:0116CE0022F9
:1019030074242FF582E43400F583E0FE642060182C
:10191300900310E0240CF582E43402F583EEF00F1B
:08192300900310E004F080D8ED
:01192B002299
:100B2B00E4F54EE54E75F003A42448F582E4341544
:100B3B00F583E493FB740193FA740293F91205DFC6
:100B4B007003020CC8E4F550F551F54F7424254F92
:100B5B00F582E43400F583E0FF7003020CC3E54E2D
:100B6B0075F003A42448F582E43415F583E493FB74
:100B7B00740193FA740293F9855082758300120500
:100B8B00F8FEEFB506087551010550020CBEE55194
:100B9B007003020CBEEE6003020CB9AD50AF4E12E7
:100BAB001674E54EB408004003020CC3900BBEF85C
:100BBB00282873020BD6020C6A020C6E020CA302DD
:100BCB000CA7020CAB020CAF020CB3AF4F12190304
:100BDB007424254FF9E43400FA7B01C0031B8B59B5
:100BEB00755A00755B00E4F55CD0031209878F55CD
:100BFB008E548D538C52E4FFFEFDFCAB55AA54A9C9
:100C0B0053A852C3120701601FAB55AA54A953A88E
:100C1B0052E47F847E1EFDFC1206611206F39003E4
:100C2B0014EFF0E4900313F0E47F587E02FDFCAB6D
:100C3B0055AA54A953A852D3120701407B90031312
:100C4B007401F0AB55AA54A953A8527F487EE8FD16
:100C5B007C001206611206F3900314EFF08059D258
:100C6B00038055AF4F121903D2107424254FF9E4AA
:100C7B003400FA7B01C0031B8B59755A00755B005E
:100C8B00E4F55CD0031209878F558E548D538C522B
:100C9B0090020AE555F08020D213801CD20E8018EA
:100CAB00D20B8014D2088010D20BD208800AE4F544
:0D0CBB0051F550054F020B57054E020B2E50
:010CC8002209
:101A0000EF540F90156393C454F0FEEFC4540F933A
:031A10002EFF2284
:10184E003012299000A5E090020CF090016EE0900D
:10185E00020DF090028E63A20190020E63A201E5CA
:0F186E007324FEFF121045C212AF73227F0022B7
:101727008F75C225E4FFE56D64056030E575B47E0D
:1017370002802EE57530E707436801056D80065383
:1017470068FEE4F56D056FE56FB40808856870D22B
:1017570025E4F56FE56825E0F568800DE57530E768
:1017670005D204A22522E4F56DE57525E0F5750F90
:05177700BF08B3A2252C
:01177C00224A
:0715FF00E0FF121A00C225F3
:10160600E4FEE56E25E0F56EEF30E736436E012029
:101616002533056DE56DB4052CE4F56D0572E572AF
:10162600B40817056CE56CAC6B7002056B14F5829B
:101636008C83E56EF00574E4F572E56E25E0F56ED3
:101646008003E4F56D0572E572B40817056CE56C68
:10165600AC6B7002056B14F5828C83E56EF0057435
:0D166600E4F572EF25E0FF0EEE64087095CC
:011673002254
:1018D900754B7E7544A0C206D20DC212D224C21124
:1018E900C201C221D200C20FC296C297E49000A5DC
:0A18F900F090016E7408F00218ABC5
:10194E0090031474B8F0E4900313F090031204F0B3
:10195E00120CC9120B2B1216CF1218D9C297C2969F
:01196E002256
:10143700E4F574900317F0A3F0A3F0AB07AA0675C1
:101447006B02756CCE856C82856B83747EF0056C40
:10145700E56C7002056B0574E4F572900315F09066
:101467000315E0C39D50498B828A83E0FF121A005F
:10147700900316EFF0900319E06F900316F0E0FF6A
:101487009004D693FE900318E06EA3F0EF9003D676
:1014970093900318F00BEBAE0270010A14F5828EDD
:1014A70083E0FFC225121606900315E004F080AF13
:1014B7009003191215FF9003181215FFD2257F7E8E
:1014C700121606D225E4FF121606D201756B0275B5
:0214D7006CCED9
:0114D90022F0
:10196F00AD0720011A900025E0FF64026004EFB478
:10197F0008097E007F261214378002D221C322D39A
:01198F002235
:101380007F020F740C2402F582E43402F5837408A2
:10139000F00F740C2403F582E43402F583E4F07C4E
:1013A000017DFDFEED1DAA0470011CF5828A83E01B
:1013B000FBAA070F740C2AF582E43402F583EBF0E4
:1013C0000EBE04E07C027D01E4FEED1DAA04700166
:1013D0001CF5828A83E0FBAA070F740C2AF582E4CD
:1013E0003402F583EBF00EBE04E07C027D05E4FEE2
:1013F000ED1DAA0470011CF5828A83E0FBAA070F89
:10140000740C2AF582E43402F583EBF00EBE04E09E
:101410007C027D09E4FEED1DAA0470011CF5828AA0
:1014200083E0FBAA070F740C2AF582E43402F583EB
:06143000EBF00EBE04E02B
:011436002293
:100E0300200603020EC7E542543865397003020F0A
:100E13000AE53924085438F539131313541F2429C8
:100E2300F8E6F570200429FF12172750D9AF701286
:100E33001A00121990056AE56AAE69700205691411
:100E4300F5828E83E570F00573E573D3948040B625
:100E5300C206D212C204D224C29690030EE0FFA3AC
:100E6300E04F603EC212900202E0FCA3E0FDA3E06B
:100E7300FEA3E02401FFE43EFEE43DFDE43CFC90E0
:100E8300020212071290028EE07002D20290031146
:100E9300E004F0D394055003020E09D202E4F002F9
:100EA3000E099001FAE0FCA3E0FDA3E0FEA3E02419
:100EB30001FFE43EFEE43DFDE43CFC9001FA120731
:100EC30012020E09202440E529647E7022300205B7
:100ED300D224C20222D200D296D206E4F573F56D73
:100EE30090030EF0A3F0F56F756902756A8E22E523
:100EF30029B4A01120050ED20090028C7402F0A335
:070F030074EEF0C207D224D6
:010F0A0022C4
:1007D700201E05D296D2972230180AC21890020B13
:1007E700E0600214F0300D03120E0320110302081B
:1007F70075E543653A6048E54324085438FFE53A10
:1008070054386F60047E0180027E00E57460047DC9
:100817000180027D00EE5D7003020986056CE56CC0
:10082700AC6B7002056B14F5828C83E0FEE5431315
:100837001313541F2431F8A6068F43157480B8C2CA
:1008470097C211C2019001FEE0FCA3E0FDA3E0FE08
:10085700A3E02401FFE43EFEE43DFDE43CFC9001FF
:10086700FE120712D221D2B2E490020BF022300618
:100877000302098630014FE543653A6003020986A2
:1008870030B208C2B290020AE0A3F030100C3090E8
:100897000990020BE06003020986056CE56CAE6BFC
:1008A7007002056B14F5828E83E0FFE54313131383
:1008B700541F2431F8A607E54324085438F5431597
:1008C70074D211D29722E543653A60030209863054
:1008D700030302098630B208C2B290020AE0A3F00D
:1008E70030100C30900990020BE06003020986205B
:1008F700001F900206E0FCA3E0FDA3E0FEA3E024B6
:1009070001FFE43EFEE43DFDE43CFC9002061207D5
:1009170012C200E54324085438F543131313541F38
:100927002431F876AAE54324085438F54313131302
:10093700541F2431F876A0E54324085438F54313AF
:100947001313541F2431F8E4F6E54324085438F50B
:1009570043131313541F2431F8E4F6E543240854D2
:1009670038F543131313541F2431F8E4F6E54324F1
:10097700085438F543131313541F2431F8E4F622AF
:0B002600302105C2217F01227F002253
:1016CF00C2A9438902900314E0FFF58C8F8A75D964
:1016DF000475DC4975DD4975DA31E4F5E9F5F9F59D
:1016EF00EBF5FB900313E0601675EC1075ED10E44D
:1016FF00F5FCF5FD754108753B10754001801375BC
:10170F00EC8075ED80E4F5FCF5FD754180F53B75DA
:08171F004010E4F5EAF5FA229E
:1018AB00E4FE900314E0658C60041216CF0EE5D9AC
:1018BB0020E2057E021216CFE58920E1051216CF34
:0D18CB007E03D28C75D840D2AED2AFAF06EE
:0118D80022ED
:03003300020F0BAE
:070F0B00C0E0C0D075D00862
:100F1200C2AF30D82AC3E5EC95EAC39541500DE53E
:100F22004025ECF5EC30D71205FC8011C3E5EC95B9
:100F320040F5EC30D70415FC800385FCFCC2D830A8
:100F4200D902C2D930DA67E53B700405FC8010E5AE
:100F52003B25ECF5EC30D70405FC800385FCFCE571
:100F6200275480F54CE52725E0F527309302052725
:100F7200200B03632701302419E527654B6006E542
:100F82002765447027753900754200852729C224D8
:100F9200801A0542E5425407701253423FE542135C
:100FA2001313541F2429F8A627752700C2DA30DB51
:100FB20049E53B700405FD8010E53B25EDF5ED307C
:100FC200D70405FD800385FDFDE543653A6029E50B
:100FD2003A54077013E53A131313541F2431F8E6F9
:100FE200F5282008036328FFE528339292E5282597
:0C0FF200E0F528053A533A3FC2DBD2AFCD
:050FFE00D0D0D0E0326C
:10100300740093F8ECC3984024701F740193F8EDB7
:10101300C39840197014740293F8EEC398400E708D
:1010230009740393F8EFC39840037F00227F0122E2
:10103300EDF8E6F008A3DFFA22EDF8E0F608A3DF07
:10104300FA22E0A363A201F0A363A201DFF475A275
:101053000022E0A363A2016DFE936CFDEE05839372
:10106300FC158363A201DFEA75A200227F00E493EB
:10107300A363A201F00F600CA3E583C2E3F58363CE
:10108300A20180EA75A20022E0A363A201F0A3E516
:1010930083C2E3F58363A201DFEE75A20022E0A31E
:1010A30063A201F0A3E583C2E4D2E3F58363A20163
:1010B300DFEC75A20022E583C2E3F583E0A363A21C
:1010C30001F0A363A201DFEE75A20022E583C2E46F
:1010D300D2E3F583E0A363A201F0A363A201DFECF3
:0F10E30075A20022F922C002C004C00612FFF05D
:0710F200D006D004D0022259
:1019B000E5D220E0FBC2AF438E2075D2028F827544
:0C19C0008300E0FFE4F5D2538EDFD2AFCD
:0119CC0022F8
:1019CD00E5D220E0FBC2AF43D2028F82758300EDDA
:0A19DD00F075D25063D250D2AF2251
:1017CB00E4FEEE247FFF1219B074242EF582E4346C
:1017DB0000F583EFF074242EF582E43400F583E0FA
:1017EB00701B74242EF582E43400F5837420F0749E
:1017FB00252EF582E43400F583E4F080040EBE80E0
:06180B00C1E49000A3F00F
:0118110022B4
:0300000002157373
:0C157300787FE4F6D8FD75817F0215BA80
:1005DF00BB010689828A83E0225002E722BBFE021A
:0905EF00E32289828A83E493224D
:1005F800BB010CE58229F582E5833AF583E02250B8
:1006080006E92582F8E622BBFE06E92582F8E22201
:0D061800E58229F582E5833AF583E493221B
:1006250075F008758200EF2FFFEE33FECD33CDCC8C
:1006350033CCC58233C5829BED9AEC99E58298400F
:100645000CF582EE9BFEED9AFDEC99FC0FD5F0D6EC
:10065500E4CEFBE4CDFAE4CCF9A88222B800C1B916
:100665000059BA002DEC8BF084CFCECDFCE5F0CB54
:10067500F97818EF2FFFEE33FEED33FDEC33FCEB8D
:1006850033FB10D703994004EB99FB0FD8E5E4F948
:10069500FA227818EF2FFFEE33FEED33FDEC33FC35
:1006A500C933C910D7059BE99A4007EC9BFCE99A29
:1006B500F90FD8E0E4C9FAE4CCFB2275F010EF2F6E
:1006C500FFEE33FEED33FDCC33CCC833C810D7076E
:1006D5009BEC9AE899400AED9BFDEC9AFCE899F8A9
:0E06E5000FD5F0DAE4CDFBE4CCFAE4C8F9223C
:0E06F300C3E49FFFE49EFEE49DFDE49CFC2218
:10070100EB9FF5F0EA9E42F0E99D42F0E89C45F04E
:0107110022C5
:0C071200ECF0A3EDF0A3EEF0A3EFF0225A
:100987008B568A578958E4F562F561F560F55FF58E
:100997005DF55EE55A455B45596012EBC0E0EAC07C
:1009A700E0E9C0E0AB59AA5AA95B12076DAB56053F
:1009B70058E558AA577002055714F91205DFF56371
:1009C700C394094007E563D3940D40E1E5636420D0
:1009D70060DBE563B42D05435E038016E563B42B46
:1009E70005435E01800C74FF2558F55874FF355791
:1009F700F557E55C60046410703FAB56AA57A958D9
:100A07001205DF64306009E55C702E755C0A802989
:100A17009000011205F8FF64786004EFB45813439F
:100A27005E01755C1074022558F558E43557F55783
:100A37008007E55C7003755C08AB560558E558AA56
:100A4700577002055714F91205DFF563C394614027
:100A57000AE563D3947A50035363DF74D02563F5B3
:100A670063C3940A400CE5639411406D74F92563E0
:100A7700F563E563D3955C5060435E0185626785E6
:100A87006166856065855F64AF5C7E00E4FCFDABF5
:100A970062AA61A960A85F12071EC8ECC8C9EDC9A0
:100AA700CAEECACBEFCBE4FCFDFEEB2563F562EEA5
:100AB7003AF561ED39F560EC38F55FAF62AE61ADDF
:100AC70060FCAB67AA66A965A864D3120701500347
:100AD700020A40435E04020A40E55E20E003E48028
:100AE7002DE55A455B4559601EAB56E55824FFF97D
:100AF700E55734FFFAEBC0E0EAC0E0E9C0E0AB59E4
:100B0700AA5AA95B12076DE55E30E20774FFFFFE84
:100B1700FDFC22E55EAF62AE61AD60AC5F30E10324
:040B27000206F322AD
:10157F00020036E493A3F8E493A34003F68001F24C
:10158F0008DFF48029E493A3F85407240CC8C3336D
:10159F00C4540F4420C8834004F456800146F6DF3C
:1015AF00E4800B01020408102040809019E7E47ECC
:1015BF00019360BCA3FF543F30E509541FFEE49331
:1015CF00A360010ECF54C025E060A840B8E493A3F8
:1015DF00FAE493A3F8E493A3C8C582C8CAC583CA23
:1015EF00F0A3C8C582C8CAC583CADFE9DEE780BEDB
:0119FF0000E7
:10071E00E88FF0A4CC8BF0A42CFCE98EF0A42CFC7A
:10072E008AF0EDA42CFCEA8EF0A4CDA8F08BF0A4F8
:10073E002DCC3825F0FDE98FF0A42CCD35F0FCEB57
:10074E008EF0A4FEA9F0EB8FF0A4CFC5F02ECD391C
:0F075E00FEE43CFCEAA42DCE35F0FDE43CFC2289
:10076D00BB011A89828A83D0F0D0E0F8D0E0F9D0AD
:10077D00E0FAD0E0FBE8C0E0C0F00207C55016E992
:10078D00F8D083D082D0E0F9D0E0FAD0E0FBC0827F
:10079D00C0830207BCBBFE16E9F8D083D082D0E03F
:0F07AD00F9D0E0FAD0E0FBC082C0830207CE2271
:0907BC00EBF608EAF608E9F62262
:0907C500EBF0A3EAF0A3E9F02235
:0907CE00EBF208EAF208E9F2225C
:00000001FF
